:0E0000000C942E010C9400000C9400000C9443
:10000E0000000C9400000C9400000C9400000C9462
:10001E0000000C9400000C9400000C9400000C9452
:10002E0000000C9400000C9400000C9400000C9442
:10003E0000000C9466010C9400000C9400000C94CB
:10004E0000000C9400000C946B010C9400000C94B6
:10005E0000000C9400000C94000004150000000039
:10006E0000000415001010101000041500181818C8
:10007E0018000415001C1C1C1C000415001E1E1E5E
:10008E001E000415001F1F1F1F000E12100C02125F
:10009E001C000F11100E01111E00000000010000C7
:1000AE0000000000000060182300E8030100545215
:1000BE00582054454136323030762E38F1320020F9
:1000CE0020524146494E41442032303137202000E3
:1000DE005452582054454136323030762E386332E1
:1000EE00002020466972737420537461727420204C
:1000FE002000545258205445413632303020762E4E
:10010E00386300202046722D545820205365747594
:10011E0070202000202020204946205365747570E1
:10012E00202020200044445320512E2047656E206D
:10013E0053657475700020204672657120545820E6
:10014E003D20783120200053617665202D2070727D
:10015E0065737320415454002020467265712054FB
:10016E0058203D2078322020004946203D20002096
:10017E00487A004564697420002031206B487A006B
:10018E003130206B487A0031303020487A003530DB
:10019E00206B487A003120206B487A0031302020C5
:1001AE00487A0031202020487A0020204B6F656667
:1001BE0066205665726966792020002E004D31202A
:1001CE00004D3220004D3320004D3420004D35209F
:1001DE000030314D487A0020316B487A0031306B57
:1001EE00487A00313030487A00353030487A005243
:1001FE0000203020202020487A002D32306442200A
:10020E0000202020202020002A3C3C3C3C3278203C
:10021E0054583E3E3E3E3E2A000080C001002D4E08
:10022E00414E00494E4600000B000400A80003009A
:10023E000803B40002001403B80001004203BA0020
:10024E0002004C032802010053032A020000F89416
:10025E00EE27EFBBF1E0F5BFE5BFF8E1A895A4B737
:10026E00A77FA4BFF0936000E09360008DE0A2E052
:10027E00BB27ED938A95E9F780E098E0A0E0B1E026
:10028E00ED930197E9F7E6E3F2E0859195910097FA
:10029E0061F0A591B59105901590BF01F001059003
:1002AE000D920197E1F7FB01F0CFE0ECEEBBEFEF23
:1002BE00EDBFE8E0EEBFC0E0D3E00C945202EA934B
:1002CE00EFE0E6BDE9911895AA93BA93EA93FA93F3
:1002DE00EFB7EA93E0917800F0917900E0931A037A
:1002EE00F0931B03A0911C03B0911D03EA0FFB1F9B
:1002FE00E0931C03F0931D033394E2E0F0E0E093EF
:10030E001803F0931903E8E0E31589F4E0911C0358
:10031E00F0911D030E94A310BE2ECF2EE0E0E093BD
:10032E001C03E0931D033324F79A9B2CAC2CE9910C
:10033E00EFBFF991E991B991A9911895AA931A93E2
:10034E000A93EA81EE0FEE0FEE0FE0640E2F10E02F
:10035E00183068F40A930395EC81FD813196EC8395
:10036E00FD833197A4910E94380E1F5FF1CF198142
:10037E00088125960895E0E0E0933E03E0933F0365
:10038E0008951A9310E0339B11E0349B1260E091B4
:10039E003E03E11709F47DC0A0913E03A33021F482
:1003AE00E0913F03E11709F46EC0123051F5F09958
:1003BE001BC0E0911403F091150360911603709128
:1003CE001703A0910003B091010380910203909155
:1003DE0003030E948410E0930003F09301036093E3
:1003EE000203709303030BC0E7E2F3E25E166F069F
:1003FE003CF4E52DF62DEC50FE4F5E2E6F2EF69A48
:10040E0042C0F09936C0A0911403B09115038091AB
:10041E00160390911703E0910003F0910103609190
:10042E000203709103030E948E10E0930003F09379
:10043E0001036093020370930303E0910403F091B0
:10044E0005036091060370910703A0910003B0911C
:10045E00010380910203909103030E94921144F4D0
:10046E00E0930003F0930103609302037093030380
:10047E0009C0E9EDFCEDE515F6052CF4E4EFF1E02D
:10048E005E1A6F0AF69AE0913E03E0933F031093D3
:10049E003E0319910895E0E8E0936100E0E0E093F7
:1004AE006100E5B9E0E3E4B9E0E0E8B9E7B9EBB93A
:1004BE00EFE0EAB9E0E0E4BDE5E0E5BDE0E0E6BD91
:1004CE00E7BDE8BDE0938000E0938100E0938500F6
:1004DE00E0938400E0938700E0938600E093890028
:1004EE00E0938800E0938B00E0938A00E093B600DF
:1004FE00E093B000E093B100E093B200E093B3005C
:10050E00E093B400E0936900EDBBE0936800E093E4
:10051E006E00E0936F00E0937000E093C100E0E89E
:10052E00E0BFE0E0E0937B00E0937F00E0937E008D
:10053E00E0ECE0937C00EBE8E0937A00E0E0ECBDC9
:10054E00E093BC00A0E10E94A70EE8E6F0E0FA936B
:10055E00EA93A0E0F3DEE0E7F0E0FA93EA93A1E09D
:10056E00EDDEE8E7F0E0FA93EA93A2E0E7DEE0E8FA
:10057E00F0E0FA93EA93A3E0E1DEE8E8F0E0FA9324
:10058E00EA93A4E0DBDEE0E9F0E0FA93EA93A5E07B
:10059E00D5DEE8E9F0E0FA93EA93A6E0CFDEE0EAF2
:1005AE00F0E0FA93EA93A7E0C9DEA0E0B0E00E9483
:1005BE005C11E53099F4E0E0EA93A0E00E94400E71
:1005CE00ACEBB0E00E94940EE0E0EA93A1E00E9452
:1005DE00400EADECB0E00E94940E64C0E0E0EA93F1
:1005EE00A0E00E94400EAEEDB0E00E94940EE0E05E
:1005FE00EA93A1E00E94400EAFEEB0E00E94940E8E
:10060E00A1E0B0E0E0EEF4E463EA70E00E9468116D
:10061E00A9E0B0E0E0E4F9E563E777E00E94681155
:10062E00A9E0B0E00E9454110E94C30FA0E0B0E018
:10063E0080E89FE40E943F10A5E0B0E00E946811A0
:10064E00A0E0B0E0E5E00E947811ADE0B0E0E0E0BF
:10065E00FAE668E170E00E946811A1E1B0E0E0E521
:10066E00FDE269E170E00E946811A5E1B0E0E0EF03
:10067E00F3EB6AE170E00E946811A9E1B0E0E0ECF2
:10068E00F6EC6DE270E00E946811ADE1B0E0E0E1E1
:10069E00FAE86EE270E00E946811A1E2B0E0E0E0DC
:1006AE000E9478111B991CC0A2E2B0E0E1E00E940A
:1006BE007811E0E0EA93A0E00E94400EA0E0B1E0E5
:1006CE000E94940EE0E0EA93A1E00E94400EA1E1A8
:1006DE00B1E00E94940EA8EEB3E00E94530F05C045
:1006EE00A2E2B0E0E0E00E9478111A9914C0F19AEB
:1006FE00E0E0EA93A0E00E94400EA0E0B1E00E948C
:10070E00940EE0E0EA93A1E00E94400EA2E2B1E076
:10071E000E94940E01C0F198199914C0F39AE0E06A
:10072E00EA93A0E00E94400EA0E0B1E00E94940E79
:10073E00E0E0EA93A1E00E94400EA3E3B1E00E9444
:10074E00940E01C0F39817DEE0917C00EE7FE093EB
:10075E007C00E0917C00ED7FE0937C00E0917C00DA
:10076E00EB7FE0937C00E0917C00E77FE0937C00E0
:10077E00A0EDB7E00E94530F589A58980E94510E60
:10078E00A2E2B0E00E945C11E13009F04FC0A1E29C
:10079E00B0E00E945C11E03051F40E94510EE0E096
:1007AE00EA93A0E00E94400EA4E4B1E009C00E94CA
:1007BE00510EE0E0EA93A0E00E94400EA6E6B1E002
:1007CE000E94940EE0E0EA93A1E00E94400EA5E59F
:1007DE00B1E00E94940E1B9919C0A1E2B0E00E94F4
:1007EE005C11F0E0309721F4A1E2B0E0E1E007C047
:1007FE00E130A0E0FA0751F4A1E2B0E0E0E00E949F
:10080E007811F69AACE2B1E00E94530F19990DC01F
:10081E00F69AF79A0E94510EA8EEB3E00E94530F7B
:10082E00A2E2B0E0E0E00E947811AACFF19BFFC0F7
:10083E00F2990DC0A1E0B0E00E945411E0930003C4
:10084E00F09301036093020370930303F29AF69BF5
:10085E0023C00E94510EE0E0EA93A0E00E94400EF9
:10086E00A7E7B1E00E94940EE0910003F09101031E
:10087E0060910203709103030E943D11A4E2B3E064
:10088E000E94E30EA4E2B3E00E94850EADE7B1E054
:10089E000E94940EF698F79AF79B5AC0E0E0EA93FE
:1008AE00A1E00E94400EA1E8B1E00E94940EA0913A
:1008BE001403B09115038091160390911703A83E6F
:1008CE00E3E0BE07E0E08E07E0E09E0721F4A7E834
:1008DE00B1E00E94940EA0911403B0911503809183
:1008EE00160390911703A031E7E2BE07E0E08E07F2
:1008FE00E0E09E0721F4AEE8B1E00E94940EA091D4
:10090E001403B09115038091160390911703A4362A
:10091E00E0E0BE07E0E08E07E0E09E0721F4A5E9E7
:10092E00B1E00E94940EA0911403B0911503809132
:10093E00160390911703A035E3ECBE07E0E08E0797
:10094E00E0E09E0721F4ACE9B1E00E94940EF79826
:10095E0018DD1B9948C0E0911403F09115036091C6
:10096E00160370911703E436A0E0FA07A0E06A07B9
:10097E00A0E07A0729F4E8EEF3E060E070E026C02C
:10098E00E83EA3E0FA07A0E06A07A0E07A0729F4A0
:10099E00E0E1F7E260E070E019C0E031A7E2FA07AB
:1009AE00A0E06A07A0E07A0729F4E0E5F3EC60E046
:1009BE0070E00CC0E035A3ECFA07A0E06A07A0E0F7
:1009CE007A0789F4E4E6F0E060E070E0E093140367
:1009DE00F09315036093160370931703F79AACE226
:1009EE00B1E00E94530F199921C0E0910003F091DC
:1009FE0001036091020370910303A1E0B0E00E9435
:100A0E006811F69AF79AE8EEF3E060E070E0E09392
:100A1E001403F093150360931603709317030E944B
:100A2E00510EA8EEB3E00E94530FF198FFCEF39B48
:100A3E004EC1F4990DC0A9E0B0E00E945411E093AC
:100A4E000003F09301036093020370930303F49A7F
:100A5E00F69B20C0E0E0EA93A0E00E94400EA8E7DB
:100A6E00B1E00E94940EE0910003F09101036091B9
:100A7E000203709103030E943D11A4E2B3E00E94B1
:100A8E00E30EA4E2B3E00E94850EADE7B1E00E9452
:100A9E00940EF698F79B5AC0E0E0EA93A1E00E940C
:100AAE00400EA1E8B1E00E94940EA0911403B09103
:100ABE0015038091160390911703A83EE3E0BE073D
:100ACE00E0E08E07E0E09E0721F4A3EAB1E00E9489
:100ADE00940EA0911403B09115038091160390917A
:100AEE001703A436E0E0BE07E0E08E07E0E09E07C5
:100AFE0021F4A5E9B1E00E94940EA0911403B091E7
:100B0E0015038091160390911703AA30E0E0BE07FB
:100B1E00E0E08E07E0E09E0721F4AAEAB1E00E9431
:100B2E00940EA0911403B091150380911603909129
:100B3E001703A130E0E0BE07E0E08E07E0E09E077D
:100B4E0021F4A1EBB1E00E94940EF7981ADC1B99E8
:100B5E0048C0E0911403F091150360911603709153
:100B6E001703E436A0E0FA07A0E06A07A0E07A07D0
:100B7E0029F4E8EEF3E060E070E026C0E83EA3E082
:100B8E00FA07A0E06A07A0E07A0729F4E1E0F0E0B6
:100B9E0060E070E019C0E130A0E0FA07A0E06A075B
:100BAE00A0E07A0729F4EAE0F0E060E070E00CC023
:100BBE00EA30A0E0FA07A0E06A07A0E07A0789F41D
:100BCE00E4E6F0E060E070E0E0931403F0931503C8
:100BDE006093160370931703F79AACE2B1E00E948C
:100BEE00530F1A9973C0E0910003F09101036091C5
:100BFE00020370910303A9E0B0E00E946811A4E61D
:100C0E00B0E00E94530FA9E0B0E00E9454110E9480
:100C1E00C30FA0E0B0E080E89FE40E943F10A5E083
:100C2E00B0E00E946811A4E6B0E00E94530F0E944B
:100C3E00510EE0E0EA93A0E00E94400EA8EBB1E076
:100C4E000E94940EA5E0B0E00E945411A0E0B0E026
:100C5E0080E89FE40E943F10A0E0B3E00E948C0F5A
:100C6E000E943811E0910003F0910103609102039C
:100C7E00709103030E943D11A4E2B3E00E94E30EC3
:100C8E00E0E0EA93A1E00E94400EACEFB0E00E94DB
:100C9E00940EA4E2B3E00E94850EA8EBBBE00E9486
:100CAE00530FF69AF79AE8EEF3E060E070E0E09307
:100CBE001403F093150360931603709317030E94A9
:100CCE00510EA8EEB3E00E94530FF398B0CEA5E0FC
:100CDE00B0E00E945411E0934803F09349036093EF
:100CEE004A0370934B03A1E0B0E00E945411E093CD
:100CFE001003F09311036093120370931303ADE08E
:100D0E00B0E00E945411E0930003F093010360934E
:100D1E000203709303037894F69B7DC1E0E0EA939F
:100D2E00A0E00E94400EA0910003B09101038091BB
:100D3E00020390910303E8EEF3E060E070E00E949E
:100D4E000811E0933A03F0933B03A0910003B09196
:100D5E0001038091020390910303E8EEF3E060E05B
:100D6E0070E00E941111DF01CB01E4E6F0E060E0DB
:100D7E0070E00E940811E0933C03F0933D03E09174
:100D8E003A03F0913B030E94AF100E943D11A4E282
:100D9E00B3E00E94E30EE0913C03F0913D030E940C
:100DAE00AF100E943D11A4E3B3E00E94E30EA4E253
:100DBE00B3E00E94850EA9ECB1E00E94940EA4E36C
:100DCE00B3E00E94850EACEDB0E00E94940EA091AF
:100DDE003A03B0913B03A83EE3E0BE0724F4ACED2A
:100DEE00B0E00E94940EF09999C0E8E0EA93A0E07A
:100DFE000E94400EE1E0F0E0E715F80521F4ABECBF
:100E0E00B1E00E94940EE2E0F0E0E715F80521F45F
:100E1E00AFECB1E00E94940EE3E0F0E0E715F805C8
:100E2E0021F4A3EDB1E00E94940EE4E0F0E0E715AA
:100E3E00F80521F4A7EDB1E00E94940EE5E0F0E094
:100E4E00E715F80521F4ABEDB1E00E94940EA091E8
:100E5E001403B09115038091160390911703A03AD5
:100E6E00E6E8BE07E1E08E07E0E09E0721F4AFED75
:100E7E00B1E00E94940EA0911403B09115038091DD
:100E8E00160390911703A83EE3E0BE07E0E08E073D
:100E9E00E0E09E0721F4A5EEB1E00E94940EA09131
:100EAE001403B09115038091160390911703A0318E
:100EBE00E7E2BE07E0E08E07E0E09E0721F4ABEE2E
:100ECE00B1E00E94940EA0911403B091150380918D
:100EDE00160390911703A436E0E0BE07E0E08E07FC
:100EEE00E0E09E0721F4A1EFB1E00E94940EA091E4
:100EFE001403B09115038091160390911703A43F2C
:100F0E00E1E0BE07E0E08E07E0E09E0721F4A7EFE8
:100F1E00B1E00E94940EACECB0E077C0ADEFB1E062
:100F2E000E94940EE52DF62D0E94AF100E943D11E9
:100F3E00AEE1B3E00E94E30E052C062821F4AFEFDC
:100F4E00B1E00E94940EA52DB62DE0E0F0E00E94D7
:100F5E00CB100E2EE7EEF3E00E94B910E02161F007
:100F6E00ABEDB0E00E94940EAEE1B3E00E94850EB0
:100F7E00ADE7B1E00E94940EA52DB62DE8EEF3E09C
:100F8E000E94BF100E2EEFE0F7E20E94B910E02192
:100F9E0061F0ACEDB0E00E94940EAEE1B3E00E94C1
:100FAE00850EADE7B1E00E94940EA52DB62DE0E0C2
:100FBE00F0E00E94C5100E2EE9E1FCEF0E94BF107A
:100FCE00E02161F0ACEDB0E00E94940EAEE1B3E032
:100FDE000E94850EADE7B1E00E94940EA52DB62DB0
:100FEE00E8E1FCEF0E94B9100E2EE1EFF8ED0E9441
:100FFE00CB10E02161F0ACEDB0E00E94940EAEE1BA
:10100E00B3E00E94850EAEE7B1E00E94940EF69812
:10101E00E1E0E0934203F79BE4C3F599D3C3E0E02C
:10102E00EA93A1E00E94400EE4E1E41519F4A8E071
:10103E00B2E002C0AFE0B2E00E94940EA7E00E94C0
:10104E00650E092C0A2801F5E7E0EA93A1E00E945B
:10105E00400EA0E00E94650EA0E00E94650EA0E08A
:10106E000E94650EA0E00E94650EA0E00E94650E33
:10107E00A0E00E94650EA0E00E94650EA0E00E9416
:10108E00650EA0E00E94650EE0E0EA93A1E00E94EA
:10109E00400EED2DFE2DE451FC4FE915FA0500F53D
:1010AE00E7E0EA93A1E00E94400EA5E00E94650EE3
:1010BE00A5E00E94650EA5E00E94650EA5E00E94C7
:1010CE00650EA5E00E94650EA5E00E94650EA5E0E6
:1010DE000E94650EA5E00E94650EA5E00E94650EB9
:1010EE00ED2DFE2DE953FC4FA92DBA2D0E94DD10DA
:1010FE000E2EED2DFE2DE451FC4F0E94D710E02157
:10110E0001F1E7E0EA93A1E00E94400EA5E00E9403
:10111E00650EA5E00E94650EA5E00E94650EA5E095
:10112E000E94650EA5E00E94650EA5E00E94650E68
:10113E00A5E00E94650EA5E00E94650EA2E00E9449
:10114E00650EED2DFE2DED55FC4FA92DBA2D0E94ED
:10115E00DD100E2EED2DFE2DE953FC4F0E94D71003
:10116E00E02101F1E7E0EA93A1E00E94400EA5E044
:10117E000E94650EA5E00E94650EA5E00E94650E18
:10118E00A5E00E94650EA5E00E94650EA5E00E94F6
:10119E00650EA5E00E94650EA5E00E94650EA0E01A
:1011AE000E94650EED2DFE2DEC56FC4FA92DBA2D8D
:1011BE000E94DD100E2EED2DFE2DED55FC4F0E94E2
:1011CE00D710E02101F1E7E0EA93A1E00E94400E82
:1011DE00A5E00E94650EA5E00E94650EA5E00E94A6
:1011EE00650EA5E00E94650EA5E00E94650EA5E0C5
:1011FE000E94650EA5E00E94650EA2E00E94650E9B
:10120E00A0E00E94650EED2DFE2DE058FC4FA92D9D
:10121E00BA2D0E94DD100E2EED2DFE2DEC56FC4F3C
:10122E000E94D710E02101F1E7E0EA93A1E00E94CD
:10123E00400EA5E00E94650EA5E00E94650EA5E099
:10124E000E94650EA5E00E94650EA5E00E94650E47
:10125E00A5E00E94650EA5E00E94650EA0E00E942A
:10126E00650EA0E00E94650EED2DFE2DE959FC4F96
:10127E00A92DBA2D0E94DD100E2EED2DFE2DE0585B
:10128E00FC4F0E94D710E02101F1E7E0EA93A1E0C4
:10129E000E94400EA5E00E94650EA5E00E94650E1C
:1012AE00A5E00E94650EA5E00E94650EA5E00E94D5
:1012BE00650EA5E00E94650EA2E00E94650EA0E0FC
:1012CE000E94650EA0E00E94650EED2DFE2DE15DE3
:1012DE00FC4FA92DBA2D0E94DD100E2EED2DFE2DE8
:1012EE00E959FC4F0E94D710E02101F1E7E0EA93A3
:1012FE00A1E00E94400EA5E00E94650EA5E00E94AE
:10130E00650EA5E00E94650EA5E00E94650EA5E0A3
:10131E000E94650EA5E00E94650EA0E00E94650E7B
:10132E00A0E00E94650EA0E00E94650EED2DFE2D40
:10133E00E050FD4FA92DBA2D0E94DD100E2EED2D81
:10134E00FE2DE15DFC4F0E94D710E02101F1E7E098
:10135E00EA93A1E00E94400EA5E00E94650EA5E072
:10136E000E94650EA5E00E94650EA5E00E94650E26
:10137E00A5E00E94650EA2E00E94650EA0E00E940C
:10138E00650EA0E00E94650EA0E00E94650EED2D98
:10139E00FE2DE153FD4FA92DBA2D0E94DD100E2E0C
:1013AE00ED2DFE2DE050FD4F0E94D710E02101F1F2
:1013BE00E7E0EA93A1E00E94400EA5E00E94650ED0
:1013CE00A5E00E94650EA5E00E94650EA5E00E94B4
:1013DE00650EA5E00E94650EA0E00E94650EA0E0DD
:1013EE000E94650EA0E00E94650EA0E00E94650EB0
:1013FE00ED2DFE2DEF54FD4FA92DBA2D0E94DD10BF
:10140E000E2EED2DFE2DE153FD4F0E94D710E02143
:10141E0001F1E7E0EA93A1E00E94400EA5E00E94F0
:10142E00650EA5E00E94650EA5E00E94650EA5E082
:10143E000E94650EA2E00E94650EA0E00E94650E5D
:10144E00A0E00E94650EA0E00E94650EA0E00E9442
:10145E00650EED2DFE2DE257FD4FA92DBA2D0E94E2
:10146E00DD100E2EED2DFE2DEF54FD4F0E94D710E8
:10147E00E02101F1E7E0EA93A1E00E94400EA5E031
:10148E000E94650EA5E00E94650EA5E00E94650E05
:10149E00A5E00E94650EA0E00E94650EA0E00E94ED
:1014AE00650EA0E00E94650EA0E00E94650EA0E011
:1014BE000E94650EED2DFE2DE458FD4FA92DBA2D7F
:1014CE000E94DD100E2EED2DFE2DE257FD4F0E94D7
:1014DE00D710E02101F1E7E0EA93A1E00E94400E6F
:1014EE00A5E00E94650EA5E00E94650EA5E00E9493
:1014FE00650EA2E00E94650EA0E00E94650EA0E0BF
:10150E000E94650EA0E00E94650EA0E00E94650E8E
:10151E00A0E00E94650EED2DFE2DE05AFD4FA92D87
:10152E00BA2D0E94DD100E2EED2DFE2DE458FD4F2E
:10153E000E94D710E02101F1E7E0EA93A1E00E94BA
:10154E00400EA5E00E94650EA5E00E94650EA5E086
:10155E000E94650EA0E00E94650EA0E00E94650E3E
:10156E00A0E00E94650EA0E00E94650EA0E00E9421
:10157E00650EA0E00E94650EED2DFE2DE15EFD4F85
:10158E00A92DBA2D0E94DD100E2EED2DFE2DE05A46
:10159E00FD4F0E94D710E02101F1E7E0EA93A1E0B0
:1015AE000E94400EA5E00E94650EA5E00E94650E09
:1015BE00A2E00E94650EA0E00E94650EA0E00E94CF
:1015CE00650EA0E00E94650EA0E00E94650EA0E0F0
:1015DE000E94650EA0E00E94650EED2DFE2DE85FC7
:1015EE00FD4FA92DBA2D0E94DD100E2EED2DFE2DD4
:1015FE00E15EFD4F0E94D710E02101F1E7E0EA9392
:10160E00A1E00E94400EA5E00E94650EA5E00E949A
:10161E00650EA0E00E94650EA0E00E94650EA0E09F
:10162E000E94650EA0E00E94650EA0E00E94650E6D
:10163E00A0E00E94650EA0E00E94650EED2DFE2D2D
:10164E00EB5FFD4FA92DBA2D0E94DD100E2EED2D54
:10165E00FE2DE85FFD4F0E94D710E02101F1E7E07B
:10166E00EA93A1E00E94400EA5E00E94650EA2E062
:10167E000E94650EA0E00E94650EA0E00E94650E1D
:10168E00A0E00E94650EA0E00E94650EA0E00E9400
:10169E00650EA0E00E94650EA0E00E94650EED2D85
:1016AE00FE2DED5FFD4FA92DBA2D0E94DD100E2EE1
:1016BE00ED2DFE2DEB5FFD4F0E94D710E02101F1C5
:1016CE00E7E0EA93A1E00E94400EA5E00E94650EBD
:1016DE00A0E00E94650EA0E00E94650EA0E00E94B0
:1016EE00650EA0E00E94650EA0E00E94650EA0E0CF
:1016FE000E94650EA0E00E94650EA0E00E94650E9D
:10170E00ED2DFE2DEC50FE4FA92DBA2D0E94DD10B1
:10171E000E2EED2DFE2DEE5FFD4F0E94D710E02117
:10172E0001F1E7E0EA93A1E00E94400EA3E00E94DF
:10173E00650EA0E00E94650EA0E00E94650EA0E07E
:10174E000E94650EA0E00E94650EA0E00E94650E4C
:10175E00A0E00E94650EA0E00E94650EA0E00E942F
:10176E00650EED2DFE2DEE53FE4FA92DBA2D0E94C6
:10177E00D1100E2EED2DFE2DEC50FE4F0E94D710E7
:10178E00E02101F1E7E0EA93A1E00E94400EA1E022
:10179E000E94650EA0E00E94650EA0E00E94650EFC
:1017AE00A0E00E94650EA0E00E94650EA0E00E94DF
:1017BE00650EA0E00E94650EA0E00E94650EA0E0FE
:1017CE000E94650EF59B09C0E0E0EA93A1E00E943D
:1017DE00400EA6E1B2E00E94940EF798E1E0E0938D
:1017EE0042030E94C801E0917A00E074E1F7F59996
:1017FE000DC0E0ECE0937C00E0917A00E064E093B1
:10180E007A00E0E0E0931803E0931903E0910803F7
:10181E00F091090360910A0370910B03A0910003EC
:10182E00B091010380910203909103030E948D11E8
:10183E0010F42D9A01C02D981B9955C0E0911403F8
:10184E00F09115036091160370911703E436A0E032
:10185E00FA07A0E06A07A0E07A0729F4E4EFF1E0C6
:10186E0060E070E033C0E43FA1E0FA07A0E06A0751
:10187E00A0E07A0729F4E8EEF3E060E070E026C01D
:10188E00E83EA3E0FA07A0E06A07A0E07A0729F491
:10189E00E0E1F7E260E070E019C0E031A7E2FA079C
:1018AE00A0E06A07A0E07A0729F4E0EAF6E861E032
:1018BE0070E00CC0E03AA6E8FA07A1E06A07A0E0E3
:1018CE007A0789F4E4E6F0E060E070E0E093140358
:1018DE00F09315036093160370931703F69AACE218
:1018EE00B1E00E94530F199914C0E42DF0E0309727
:1018FE0029F4E4E14E2EF79A2C9A07C0E431A0E0C9
:10190E00FA0739F44424F79A2C98ACE2B1E00E941D
:10191E00530F1A9915C0E0E0F099E1E0E03011F4B0
:10192E00F09A03C0E13061F4F098F69AE1E0E093AA
:10193E004203ACE2B1E00E94530F0E94510EF79A9F
:10194E00329986C0E72DF82DE130A0E0FA0799F420
:10195E00E2E0F0E07E2E8F2EE0910003F091010385
:10196E006091020370910303ADE0B0E00E94681134
:10197E00A1E1B0E05BC0E230A0E0FA0799F4E3E049
:10198E00F0E07E2E8F2EE0910003F0910103609126
:10199E00020370910303A1E1B0E00E946811A5E17A
:1019AE00B0E044C0E330A0E0FA0799F4E4E0F0E0E0
:1019BE007E2E8F2EE0910003F091010360910203C1
:1019CE0070910303A5E1B0E00E946811A9E1B0E0B7
:1019DE002DC0E430A0E0FA0799F4E5E0F0E07E2EA9
:1019EE008F2EE0910003F09101036091020370913C
:1019FE000303A9E1B0E00E946811ADE1B0E016C0AA
:101A0E00E530A0E0FA0721F5E1E0F0E07E2E8F2E22
:101A1E00E0910003F09101036091020370910303C2
:101A2E00ADE1B0E00E946811ADE0B0E00E9454114B
:101A3E00E0930003F093010360930203709303039A
:101A4E00F69AACE2B1E00E94530F0E94510EF79A43
:101A5E00E0E0319BE1E00E2EA0E0F599A1E0E0E0A0
:101A6E000E94B410E02129F0F59AE1E0E0934203E0
:101A7E00F79AE0E03199E1E00E2EA0E0F599A1E0B1
:101A8E00E1E00E94B410E021F9F0F598F79AE7E052
:101A9E00EA93A1E0EED0A0E00E94650EA0E00E94C5
:101AAE00650EA0E00E94650EA0E00E94650EA0E00B
:101ABE000E94650EA0E00E94650EA0E00E94650ED9
:101ACE00A0E0FCD0A0E0FAD0A0914203A13009F032
:101ADE0094C0F894F59B0BC0E0910003F0910103C4
:101AEE0060910203709103030E94AA102BC0F09B19
:101AFE0017C0E0911003F0911103609112037091E1
:101B0E001303A0910003B091010380910203909101
:101B1E0003030E948910E52DF62D0E94AF1010C010
:101B2E00E0911003F0911103609112037091130371
:101B3E00A0910003B09101038091020390910303E1
:101B4E000E948410E0930C03F0930D0360930E0338
:101B5E0070930F03E0E0E0934703E0914803F091A8
:101B6E00490360914A0370914B03A0910C03B0910D
:101B7E000D0380910E0390910F030E9444110E9459
:101B8E00F10FA3E4B3E00E948A0F0E9438115A9A13
:101B9E005A98E0E0E0934103A0914103A53028F567
:101BAE00E0E0E0934003A0914003A830C0F4E09140
:101BBE004103F0E0ED5BFC4F1080E0914003A1E0AB
:101BCE000E949B10E12111F4599801C0599A5B9A19
:101BDE005B98E0914003EF5FE0934003E4CFE09128
:101BEE004103EF5FE0934103D7CF59985A9A5A9821
:101BFE00E0E0E0934203789467CF0C949306FFCF16
:101C0E00AA93E881E07111F05D9A01C05D98E881B8
:101C1E00E07211F02F9A01C02F98E881E07411F054
:101C2E002E9A01C02E98E881E07811F05C9A01C0DE
:101C3E005C988DE08A95F1F75E9A8DE08A95F1F7C2
:101C4E005E988DE08A95F1F7B5C0AA93A881D8DF8A
:101C5E00E881E295E883A881D3DF85E88A95F1F7DC
:101C6E00A9C0AA93A981F1DF289AA881EEDF28984E
:101C7E000FC0AA93E881F0E0E45BFC4FE081A981FC
:101C8E00AE0FE3DFE981E0935003E881E093510367
:101C9E0022960895A2E0D9DFA3E0B0E00E94530F90
:101CAE00ACE0D3DFA1E0D1DFA3E0B0E00E94530FA0
:101CBE00E0E0E0935103E09350030895AA93A881C6
:101CCE00AA3031F0E0915203A0915003AE1760F0AC
:101CDE00E0E0EA93A0915103AF5FA0935103C9DFF7
:101CEE00A881AA3009F466C0E0915003EF5FE0933B
:101CFE005003289AA881A9DF28985CC0BA93AA93AA
:101D0E001A93A981BA81ED91A983BA831E2FE0306F
:101D1E0019F0A12FD3DFF5CF10C0BA93AA931A935F
:101D2E00E981FA813196E983FA833197E4911E2F86
:101D3E00E03019F0A12FC2DFF3CF1881239608955A
:101D4E00AA93559A279A269A549A569A209A579A4F
:101D5E005E9828985F98E881E0935203E058E093EC
:101D6E004E03E881E054E0934F03A4E1B0E00E94FB
:101D7E00530FA0E345DF88EC90E00197F1F7A0E365
:101D8E003FDF88EC90E00197F1F7A0E339DF88ECB4
:101D9E0090E00197F1F7A0E233DF88EC90E0019735
:101DAE00F1F7A8E252DFA4E050DFA5E84EDFA6E08F
:101DBE004CDF70DF21960895BA93AA9324971A9355
:101DCE000A93E0E0FAEC6AE97BE3EA83FB836C8337
:101DDE007D8300E0AB85AA2392F4E885F9856A85B8
:101DEE007B850E949310E887F9876A877B87AE818F
:101DFE00BF811196AE83BF831197EDE2EC93EA811A
:101E0E00FB816C817D81A885B9858A859B850E9421
:101E1E00E3101E2F103071F4003061F4AA81BB81E3
:101E2E008C819D81A130E0E0BE07E0E08E07E0E00E
:101E3E009E0751F4AE81BF811196AE83BF83119779
:101E4E00E12FE05DEC9301E0EA81FB816C817D8105
:101E5E00A885B9858A859B850E940D11E887F9872B
:101E6E006A877B87AA81BB818C819D81EAE0F0E045
:101E7E0060E070E00E94E310EA83FB836C837D8355
:101E8E000E94891109F0BBCFAE81BF81E0E0EC93D7
:101E9E00198108812C960895109639F080ED97E0FF
:101EAE000197F1F7A8951197C9F70895552342F4B4
:101EBE00503811F4E0FF04C03196691F791F6BF0A2
:101ECE0050E8572711F45F9373C05F3F31F0660FF0
:101EDE00000C57956795752F08955F9300200AF0B3
:101EEE0073C06CC050E8192E1522880F991F9527C4
:101EFE00550F879550E8072E0522660F771F752719
:101F0E00550F67950895689401C0E8945F93F2DFCA
:101F1E00703818F07F3F08F44BC056E1571BAAF4F7
:101F2E00519558300EF4593030F0EFEFFFEF6FEF60
:101F3E007FE777F91AC077275523B9F0EE0FFF1F09
:101F4E00661F771F5A95D1F710C07727583028F0A3
:101F5E00EF2FF62F672F5850F9CF552331F0769586
:101F6E006795F795E7955A95D1F700200AF4D4D0E6
:101F7E005F910895689401C0E89430976040704076
:101F8E00B1F0002426F0772312F40094C5D0172E5A
:101F9E007EE1112032F07A95EE0FFF1F661F111CA5
:101FAE00F9CFEF2FF62F612D5F938ADF5F910895A2
:101FBE00EE27FF27662777275F910895EFEFFFEF54
:101FCE006FE77FEF5F910895EFEFFFEF6FE77FE72A
:101FDE005F9108955F9386DF703851F3903841F327
:101FEE0001240894791F23F41CF300203AF3ECCF5C
:101FFE000F921F932F933F934F93112722279927C9
:10200E00689FA0018F9F302D410D591F6B9F300D82
:10201E00411D591F8E9F27D0BF9F25D06A9F23D069
:10202E00BE9F1DD0AF9F1BD0AE9F110D291F391F14
:10203E00491F591FE32FF42F652F522F4F913F91B8
:10204E002F911F910F9066232AF0550FEE1FFF1F41
:10205E00661F02C073954BF229DF5F910895100D34
:10206E00211D391F02C0200D311D491F591F089512
:10207E005F9338DF703821F411200AF49FCFA4CF7C
:10208E00903809F495CF01240894970B1BF4D4F3E0
:10209E000020F3CF792F1F932F933F934F9311244B
:1020AE001127222733274427552790E2AE17BF0763
:1020BE008607410730F0AE1BBF0B860B410B089411
:1020CE0001C08894551F221F331F111CAA1FBB1F4E
:1020DE00881F441F9A9551F7F901612D4F913F9139
:1020EE002F911F91662332F0550FEE1FFF1F661FB3
:1020FE007A9543F2DBDE5F910895EA0FFB1F681FAE
:10210E00791F0895AE0FBF1F861F971F0895EA1BF4
:10211E00FB0B680B790B0895F09560957095E19522
:10212E00FF4F6F4F7F4F0895EE230E2EEA2F19F0BB
:10213E00EE0F0A94E9F70895F695E795F695E7956B
:10214E00F695E7950895EE0FFF1F661F771F08950A
:10215E006F2F660F660B762F0895EA17E1E009F0F0
:10216E00EE270895EA17FB07E1E00CF4EE27089539
:10217E00AE17BF07E1E00CF4EE270895AE17BF07C8
:10218E00E1E00CF0EE270895EA17FB07E1E00CF012
:10219E00EE270895AE17BF07E1E008F4EE27089585
:1021AE00AE17BF07E1E008F0EE270895EA17FB0728
:1021BE00E1E008F0EE2708953F934F935F930024DC
:1021CE0011244427552730E2AA0FBB1F881F991FE1
:1021DE00001C111C441F551F0E1A1F0A460B570BCD
:1021EE0028F40E0E1F1E461F571F01C0A1603A9500
:1021FE0059F7FD01BC01D001CA015F914F913F918A
:10220E0008951CD0D9DF0EF487DF0895D5DFFD01C8
:10221E00BC010895E89497FF09C0A095B0958095EC
:10222E009095AF5FBF4F8F4F9F4F689477FD74DFD0
:10223E00C3DFFD01BC010EF46FDF0895E89477FF54
:10224E0002C06ADF689497FF0BC00024A095B0957A
:10225E00809590951196801D901D00F8039400FABC
:10226E000895ED93FD936D937C9308957A936A93FD
:10227E00FA93EA930895689401C0E89401D07DDE44
:10228E00182E862F612D192E972F712D1B2EBF2FD5
:10229E00F12D1A2EAE2FE12D0895129602D0BF0108
:1022AE001297119602D0FE2F1197F999FECFFF9338
:1022BE00FFB7F894A1BDB2BDF89AE0B5FFBFFF918C
:1022CE00089507D012960F01FB0103D0F00112976B
:1022DE00089507D01196EF93EF2F03D0EF9111973A
:1022EE000895F99B02C0A895FCCF9FB7F894A1BDA5
:1022FE00B2BDF89A80B5E81719F0E0BDFA9AF99ACE
:10230E009FBF08953097604070400895EA17FB070D
:10231E00680779070895AE17BF07860797070895D0
:00000001FF
